:02000000682F67
:1000060083160313981809280000032883126D0825
:040016009900080045
:10001A0083120313FB01FA01F9018030F800F10C95
:10002A00F00C031C21287408F90775080318750FCA
:10003A00FA070318FB0A0310F01F29287408FA07A5
:10004A0075080318750FFB07FB0CFA0CF90CF80C72
:10005A00031C14287B08F3007A08F2007908F100DF
:06006A007808F000080018
:1000700083120313FB01FA01F901F801A001730DCA
:10008000F80D7408F8027508031C750FF90276085C
:10009000031C760FFA027708031C770FFB0200019E
:1000A000031C0130A002F30D0730FC00730DF80DA6
:1000B000F90DFA0DFB0DA00D7408731C7128F802E0
:1000C0007508031C750FF9027608031C760FFA02F7
:1000D0007708031C770FFB020001031C0130A0020C
:1000E0008228F80775080318750FF90776080318B2
:1000F000760FFA0777080318770FFB07000103183C
:100100000130A007F30DFC0B5628720DF80DF90D08
:10011000FA0DFB0DA00D7408731CA028F8027508D9
:10012000031C750FF9027608031C760FFA02770894
:10013000031C770FFB020001031C0130A002B12851
:10014000F80775080318750FF90776080318760F76
:10015000FA0777080318770FFB070001031801302F
:10016000A007F20D0730FC00720DF80DF90DFA0D25
:10017000FB0DA00D7408721CCF28F8027508031C33
:10018000750FF9027608031C760FFA027708031C34
:10019000770FFB020001031C0130A002E028F807E2
:1001A00075080318750FF90776080318760FFA0714
:1001B00077080318770FFB07000103180130A00729
:1001C000F20DFC0BB428710DF80DF90DFA0DFB0DB5
:1001D000A00D7408721CFE28F8027508031C750F28
:1001E000F9027608031C760FFA027708031C770FD2
:1001F000FB020001031C0130A0020F29F80775085B
:100200000318750FF90776080318760FFA077708B1
:100210000318770FFB07000103180130A007F10D49
:100220000730FC00710DF80DF90DFA0DFB0DA00D56
:100230007408711C2D29F8027508031C750FF9024A
:100240007608031C760FFA027708031C770FFB026F
:100250000001031C0130A0023E29F80775080318AD
:10026000750FF90776080318760FFA077708031851
:10027000770FFB07000103180130A007F10DFC0BFD
:100280001229700DF80DF90DFA0DFB0DA00D740873
:10029000711C5C29F8027508031C750FF9027608B9
:1002A000031C760FFA027708031C770FFB0200018C
:1002B000031C0130A0026D29F80775080318750F9B
:1002C000F90776080318760FFA0777080318770FEF
:1002D000FB07000103180130A007F00D0730FC00F8
:1002E000700DF80DF90DFA0DFB0DA00D7408701CC2
:1002F0008B29F8027508031C750FF9027608031C98
:10030000760FFA027708031C770FFB020001031C2B
:100310000130A0029C29F80775080318750FF9072A
:1003200076080318760FFA0777080318770FFB078C
:10033000000103180130A007F00DFC0B70297018A4
:10034000AF297408F80775080318750FF9077608C0
:100350000318760FFA0777080318770FFB070800D2
:0E0360008312031368088A00670882000800F1
:10036E00031CBF2983120313051485108514C42999
:0C037E008312031305108510851408007D
:10038A0083160313981690308312980083168614E6
:10039A00061183128C1ED4291A08F000CE290800EF
:1003AA009A01981718168C1ED8291A08E900981C61
:0803BA000800181208000800F9
:1003C200B03083120313E2001630E300D230E400AF
:1003D200E501061086150612861606138613080016
:1003E20083120313EC016A0884000008EB006B0817
:1003F200003A0319062A6B08ED000320EC0A6C0888
:0C0402006A0784000008EB00F8290800DD
:10040E00831203137008F100F0010830FC0071082C
:10041E00F40C0318162AFC0B0F2AF10100340310FA
:10042E001B2AF40C0318F107F10CF00CFC0B182A24
:02043E000800B4
:10044000831203132230FC00F801F901FA01FB01C9
:10045000FC030319562A0310FB0CFA0CF90CF80CD8
:10046000F30CF20CF10CF00C031C282AFC0303190A
:10047000482A7408F80775080318750FF9077608F5
:100480000318760FFA0777080318770FFB072C2A53
:100490007408F80775080318750FF907760803182C
:0E04A000760FFA0777080318770FFB0708009E
:1004AE006400293083120313EA00F121D521690873
:1004BE00493A031D642AD521652A572A6908463A06
:1004CE00031D6D2AD521D521D5216E2A572AE60185
:1004DE006608203C031C7B2AD5216608A03E8400BA
:1004EE0069088000E60A6F2A83163708313A031D21
:1004FE00832A83120512852A83120516831638085D
:10050E00353A031D8E2A01308312E100902A8312A0
:10051E00E10183163808343A031D992A01308312FB
:10052E00BF009B2A8312BF01831640083B3A031D6E
:10053E00A32A83128515A62A83128511E121303054
:10054E00831620028312BB00BC01031CBC030030C7
:10055E00BC1BFF30BD00BE003B08F0003C08F100A4
:10056E003D08F2003E08F3008030F4009630F500AE
:10057E009830F6000030F70020227008BB0071089A
:10058E00BC007208BD007308BE0030308316210215
:10059E008312B700B801031CB8030030B81BFF303C
:1005AE00B900BA003708F0003808F1003908F20037
:1005BE003A08F3004030F4004230F5000F30F600F8
:1005CE000030F70020227008B7007108B8007208DA
:1005DE00B9007308BA003030831622028312C000AD
:1005EE00C101031CC1030030C11BFF30C200C30098
:1005FE004008F0004108F1004208F2004308F30001
:10060E00A030F4008630F5000130F6000030F7001F
:10061E0020227008C0007108C1007208C200730861
:10062E00C3003030831623028312C800C901031C95
:10063E00C9030030C91BFF30CA00CB004808F000C8
:10064E004908F1004A08F2004B08F3001030F4009C
:10065E002730F500F601F70120227008C800710856
:10066E00C9007208CA007308CB003030831624020A
:10067E00F000F101031CF10370088312C60071082B
:10068E00C700E830F4000330F5000D207008C600F6
:10069E007108C700303083162502F000F101031CEB
:1006AE00F10370088312C4007108C5006430F400B1
:1006BE000030F5000D207008C4007108C500303000
:1006CE0083162602F00070088312B2000A30F4007E
:1006DE0007227008B200303083162702F90079081D
:1006EE008312B1007908B1003B08F1003C08F2001A
:1006FE003D08F3003E08F4003708F10738080318E8
:10070E00380FF20739080318390FF3073A080318A0
:10071E003A0FF4074008F10741080318410FF2079A
:10072E0042080318420FF30743080318430FF40758
:10073E007108F5007208F6007308F7007408F800E7
:10074E004808F50749080318490FF6074A08031821
:10075E004A0FF7074B0803184B0FF8074608F1002E
:10076E004708F200F301F4017508F1077608031843
:10077E00760FF20777080318770FF3077808031838
:10078E00780FF4074408F5004508F600F701F80164
:10079E007108F50772080318720FF607730803182D
:1007AE00730FF70774080318740FF8077008F10039
:1007BE00F201F301F4017508F10776080318760FBC
:1007CE00F20777080318770FF30778080318780FE6
:1007DE00F4077908AD00AE01AF01B0017108AD07A5
:1007EE0072080318720FAE0773080318730FAF0762
:1007FE0074080318740FB00700303002031D112C5B
:10080E0015302F02031D112C35302E02031D112C15
:10081E00AF302D020318242C3008013C031D212C6F
:10082E002F08D93C031D212C2E08053C031D212C1D
:10083E002D08C03C0318242C032C00303002031D5D
:10084E00322C15302F02031D322C5C302E02031D6C
:10085E00322CC0302D02031C4F2C3008003C031DDF
:10086E00422C2F08213C031D422C2E08913C031DC7
:10087E00422C2D08BF3C031C4F2C3308E4000610FD
:10088E00861506128612061386132030B600FD2D2D
:10089E0000303002031D5D2C21302F02031D5D2C14
:1008AE0091302E02031D5D2CC0302D02031C7A2CBC
:1008BE003008003C031D6D2C2F082D3C031D6D2CA4
:1008CE002E089F3C031D6D2C2D08AF3C031C7A2C6B
:1008DE003508E400061486150612861606138613CE
:1008EE001030B600FD2D00303002031D882C2D3047
:1008FE002F02031D882CC6302E02031D882CC030FB
:10090E002D02031CA52C3008003C031D982C2F082B
:10091E00443C031D982C2E08833C031D982C2D0857
:10092E000F3C031CA52C3508E40006108615061294
:10093E008616061386131030B600FD2D00303002D9
:10094E00031DB32C44302F02031DB32CAA302E02EC
:10095E00031DB32C20302D02031CD02C3008003C7C
:10096E00031DC32C2F085B3C031DC32C2E08663CB5
:10097E00031DC32C2D086F3C031CD02C3408E4003F
:10098E000614861506168616061386130830B6004C
:10099E00FD2D00303002031DDE2C5B302F02031DB7
:1009AE00DE2C66302E02031DDE2C70302D02031C51
:1009BE00FB2C3008003C031DEE2C2F08893C031D38
:1009CE00EE2C2E082D3C031DEE2C2D082F3C031C67
:1009DE00FB2C5C08E4000610861506168616061318
:1009EE0086130830B600FD2D00303002031D092D90
:1009FE0089302F02031D092D2D302E02031D092DC6
:100A0E0030302D02031C262D3008003C031D192DFD
:100A1E002F08B63C031D192D2E08F33C031D192D6E
:100A2E002D08EF3C031C262D5B08E40006148615EA
:100A3E0006128612061786130430B600FD2D0030FE
:100A4E003002031D342DB6302F02031D342DF3302A
:100A5E002E02031D342DF0302D02031C512D3008B3
:100A6E00013C031D442D2F080A3C031D442D2E0866
:100A7E00E03C031D442D2D084F3C031C512D5A08FC
:100A8E00E400061086150616861206178613043025
:100A9E00B600FD2D01303002031D5F2D0A302F02EE
:100AAE00031D5F2DE0302E02031D5F2D50302D02F1
:100ABE00031C7C2D3008013C031D6F2D2F08313C8B
:100ACE00031D6F2D2E08053C031D6F2D2D08EF3CC9
:100ADE00031C7C2D5D08E400061486110616861292
:100AEE00061386130430B600FD2D01303002031DAF
:100AFE008A2D31302F02031D8A2D05302E02031D43
:100B0E008A2DF0302D02031CA72D3008013C031D49
:100B1E009A2D2F085E3C031D9A2D2E08CC3C031DEA
:100B2E009A2D2D08AF3C031CA72D6008E400061477
:100B3E00861106168612061386130430B600FD2D96
:100B4E0001303002031DB52D5E302F02031DB52D71
:100B5E00CC302E02031DB52DB0302D02031CD22D2C
:100B6E003008013C031DC52D2F088C3C031DC52DDF
:100B7E002E08933C031DC52D2D086F3C031CD22D52
:100B8E005F08E400061086110616861606178613F1
:100B9E000430B600FD2D01303002031DE02D8C30E7
:100BAE002F02031DE02D93302E02031DE02D703019
:100BBE002D02031CFD2D3008013C031DF02D2F08C6
:100BCE00D83C031DF02D2E08DE3C031DF02D2D0804
:100BDE00B03C031CFD2D5E08E400061086110612C3
:100BEE008612061386170430B600FD2D051E2A2E1A
:100BFE001030F4002730F500F601F7012D08F00053
:100C0E002E08F1002F08F2003008F3007408F002ED
:100C1E007508031C750FF1027608031C760FF2029D
:100C2E007708031C770FF3023608F400F501F6017E
:100C3E00F70120227008AD007108AE007208AF00F7
:100C4E007308B000742E6108013A0319332E3F0861
:100C5E00013A0319332E5E2E8C30F4002330F5004A
:100C6E00F601F7012D08F0002E08F1002F08F20012
:100C7E003008F3007408F0027508031C750FF102BA
:100C8E007608031C760FF2027708031C770FF30227
:100C9E003608F400F501F601F70120227008AD00C8
:100CAE007108AE007208AF007308B000742E2D08E4
:100CBE00F0002E08F1002F08F2003008F30036087D
:100CCE00F400F501F601F70120227008AD0071085D
:100CDE00AE007208AF007308B0001030F400273079
:100CEE00F500F601F7012D08F0002E08F1002F088F
:100CFE00F2003008F30038207008D4007108D500D7
:100D0E000030F200F300A030F4008630F500013020
:100D1E00F6000030F70020227008D0007108D100D4
:100D2E007208D2007308D3000A30F400F501F60100
:100D3E00F70138207008D0007108D1007208D20077
:100D4E007308D3002D08F4002E08F5002F08F600C6
:100D5E003008F7007008F4027108031C710FF502D9
:100D6E007208031C720FF6027308031C730FF7024E
:100D7E007408CC007508CD007608CE007708CF0039
:100D8E000A30F000F101F201F30120228830F40064
:100D9E000130F500F601F70138207008D600710811
:100DAE00D7005408E2005508E3007008E50008007B
:100DBE0083120313E209E309E409E5090515E601C7
:100DCE0066080F3C031CF62E08306602031CF02E3C
:100DDE000511E30CE20CE313B721E60AE72EE60158
:100DEE006608073C031C002FE40CE413B721E60A47
:100DFE00F72EE6016608073C031C0A2FE50D651069
:080E0E00B721E60A012F0800DC
:100E16000730831203139F008316850182308600F4
:100E26000E308100831205158514051405168515E7
:100E36008230FC00DD30FD00FD0B1F2FFC0B1F2F49
:100E4600000000008511E101BF011030D8002730F5
:100E5600D900D330B300D230B500D630B400D63086
:100E6600DC00D430DB00D430DA00D430DD00D430FE
:100E7600E000D430DF00D430DE000C308316990059
:100E86001815C5218230FC00DD30FD00FD0B492F11
:0A0E9600FC0B492F000000000800CB
:100EA00083120313861B582F2530EA00F1215B2F94
:080EB0002130EA00F1210800E5
:100EB800B0218A110A128000840AE70A0319E80A95
:080EC800F003031D5C2F08007C
:100ED000523083120313A1005830A2003B30A3000C
:100EE000A4015430A5005830A6003B30A700A8014B
:100EF0004930A9004630AA003B30AB00AC010B27BB
:100F00006400E121DF2657225027DF26832F872F19
:02400E0025216A
:00000001FF
